:100000000C944A000C9469000C9469000C946900EB
:100010000C9469000C9469000C9469000C946900BC
:100020000C9469000C9469000C9469000C946900AC
:100030000C9469000C9469000C9469000C9469009C
:100040000C9469000C9469000C9469000C9469008C
:100050000C9469000C9469000C9469000C9469007C
:100060000C9469000C9469000C9469000C9469006C
:100070000C9469000C9469000C9469000C9469005C
:100080000C9469000C9469000C9469000C9469004C
:100090000C94690011241FBECFEFD0E1DEBFCDBFAD
:1000A00011E0A0E0B1E0E2E0F2E000E00BBF02C04E
:1000B00007900D92A030B107D9F711E0A0E0B1E0B0
:1000C00001C01D92A030B107E1F70E94A7000C9477
:1000D00000010C940000CF93DF93CDB7DEB7E2E2CE
:1000E000F0E01082E1E2F0E01082E5E2F0E0108260
:1000F000E4E2F0E01082E8E2F0E01082E7E2F0E013
:100100001082EBE2F0E01082EAE2F0E088E0808327
:10011000EEE2F0E01082EDE2F0E080E18083E1E3E6
:10012000F0E01082E0E3F0E01082DF91CF910895DB
:10013000CF93DF93CDB7DEB7EF93E8E1E0936000B4
:10014000E7E0E0936000EF91DF91CF910895CF93C6
:10015000DF93CDB7DEB724970FB6F894DEBF0FBE9E
:10016000CDBF0E9498000E946B00A895A895AEE2B2
:10017000B0E0EEE2F0E0808180618C9319821A8217
:100180001B821C820BC089819A81AB81BC81019644
:10019000A11DB11D89839A83AB83BC8389819A8118
:1001A000AB81BC8180342CE9920720E0A20720E0DB
:1001B000B20748F3A895AEE2B0E0EEE2F0E090813D
:1001C0008FEE89238C9319821A821B821C820BC0AA
:1001D00089819A81AB81BC810196A11DB11D898362
:1001E0009A83AB83BC8389819A81AB81BC81803443
:1001F0002CE9920720E0A20720E0B20748F3B6CF2F
:02020000FFCF2E
:00000001FF
